:03000000023D8F2F
:0C3D8F0078FFE4F6D8FD75815F023DD698
:102381000A53746172743A20004950436F6E6E654E
:1023910063745245510A00444843502D4F4B0A0083
:1023A1004950436F6E6E65637400C0E4E0EFF2E57F
:1023B100F020D1E8EDEAEEEC4950284343290A0028
:1023C100C2E5F0F1E8FF20495020ECEEE4F3EBFF29
:1023D1003A20322E3420EEF22032302E31312E329C
:1023E1003030350A00C4E0F2E020F1EEE7E4E0ED40
:1023F100E8FF3A20004F6374203331203230303609
:1024010000200031343A30383A3031000A000A50A5
:10241100524F473A20202020202020202020202019
:1024210020202020202020202020202020202020AB
:10243100202020202020202020202020202020209B
:10244100202020202020202020202020202020208B
:102451002020202020202020200A0044756D705863
:1024610020202020203030203031203032203033E5
:10247100203034203035203036203037203038209D
:102481003039203041203042203043203044203048
:10249100452030460A003A200044756D70442020E2
:1024A1002020203030203031203032203033203095
:1024B1003420303520303620303720303820303944
:1024C100203041203042203043203044203045200C
:1024D10030460A00457272206B65790052642065AE
:1024E1006570726F6D0A005264204D454D0A0044BB
:1024F100656275674950204F4E0A004465627567F1
:102501004950204F46460A00446562756755736518
:1025110072204F6E0A0044656275675573657220BB
:102521004F46460A0044656275674D7367204F6EDA
:102531000A0044656275674D7367204F46460A007D
:10254100436F6E666967206C6F636B210A00577277
:1025510020656570726F6D0A002053617665206594
:102561006570726F6D210A00457272204D414321E1
:10257100004C6F61643E3E0057616974526573742B
:1025810061727421004E4F4950004C494E4B434FEC
:102591004E5452005452415353004652004E4F4C38
:1025A100494E4B00494E490000FF2586FF258BFF10
:0E25B1002595FF259BFF259EFF25A5FF25A94B
:0645AC00015C00015A0051
:10456A00C2AFC28E758900438910758BFF758DB7EE
:07457A00D2ABD28ED2AF22BA
:03001B00023CF9AB
:103CF900C0E0C083C082C0D0C2AFC28E758BFF75D1
:103D09008DB720060675A61E75A6E1055AD202E5ED
:103D19005C6002055C055FE55F540F7053D20DE5E9
:103D29005F543F7014D200906EB5E0600C04F0E06F
:103D3900D394B44004C2AF80FE906EB0E060020438
:103D4900F0E55BD394014002155B9069ADE0600238
:103D590014F0906EB6E0D394014003E014F03005FE
:103D690002055DE55ED394644004D2068002055ED7
:103D7900E559D3940140021559D28ED2AFD0D0D093
:063D890082D083D0E0327D
:1043F600E4FFFEFD74832DF582E4346BF583E02F34
:10440600FFE43EFE0DBD10ECE4FD74D82DF582E40C
:104416003469F583E0FC2FFFE43EFEEC60040DBD3D
:0244260080E82C
:014428002271
:10097400C291C290C2B5C20A7D027C007F071245B3
:10098400178F3CE53C646060097D017F6012448EF2
:10099400D20AE4FDFC7F0B1245178F3CE53C30E6A0
:1009A400097D04E4FF1244B2D20A7D017C007F0772
:1009B4001245178F3CE53C7008FD7FFF12448ED230
:1009C4000A300A03126000C2AFC288D2A8C2AA12B7
:1009D4004025C291D290D2AF1243F61227D1D2B59C
:1009E400D291C290906EB1121FD700000000E47F34
:1009F400207E4EFDFC906EB1E0F8A3E0F9A3E0FA8E
:100A0400A3E0FBC3121F845027906EB1E0FCA3E067
:100A1400FDA3E0FEA3E0FFE4FAF9F8EF2401FFEA06
:100A24003EFEE93DFDE83CFC906EB1121FCB80BE5A
:100A3400D291D290123864C206C291D290124286E8
:100A4400D291C290906B81E0C3940350037403F07D
:100A5400D20CD20BD20AD293200A077E237F8112B2
:100A6400377FE4906DA1F012456AC2AF755B01A3B4
:100A7400F0C207C208D2AF75A70775A61E75A6E116
:100A8400124534D291D290906EB1121FD70000005B
:100A940000E47F207E4EFDFC906EB1E0F8A3E0F907
:100AA400A3E0FAA3E0FBC3121F845027906EB1E0C9
:100AB400FCA3E0FDA3E0FEA3E0FFE4FAF9F8EF24D1
:100AC40001FFEA3EFEE93DFDE83CFC906EB1121FD9
:100AD400CB80BEC291C290200A19AF3C7E007D0338
:100AE400123943E4FF123BA97E6B7FA1E4FB7D0135
:100AF400123A21906EB5E060037401F0E49069ADA0
:100B0400F0A37455F0A37481F0E4F55DE4F55E9010
:100B140069ADE070031225BF906EB6E0B401119088
:100B240080007410F0E4906EB6F0D20AD20BD20CAE
:100B3400E55DD39403402D908002E4F0908001F0B1
:100B4400908000F0E55DD3940540037401F0E55D09
:100B5400D3940A400FE4F55DC203906DA2F0755B77
:100B6400011242869080A0E070077FCB7E03123F83
:100B7400259080B8E07003123C579080D0E0701448
:100B8400300E11906EAC74FFF0906B75E0FEA3E034
:100B9400FF12409A908000E07013300710123673F1
:100BA400906B5DEFF0D39400400312112690800205
:100BB400E07006908000E06005D205020B10C205CB
:100BC400E4F55D9069ADE06003020B103009151285
:100BD4003059906B5DEFF0D394004008300105E08C
:100BE400FF124581200803020DEF122EDC906B5D8D
:100BF400EFF07003020B10906EB5E060037401F027
:100C0400906BA1E054BF247F7003020CC3147003E3
:100C1400020CA424026003020D9A200A077E237F9B
:100C24008A12377F906B79E0FF7006906B7DE060ED
:100C340055906EACE0FEB50722A3E0FF906B7AE01E
:100C4400B50718906EAEE0FF906B7BE0B5070C9093
:100C54006EAFE0FF906B7CE06F602B906B7DE06E7D
:100C64007035906EADE0FF906B7EE0B50729906E15
:100C7400AEE0FF906B7FE0B5071D906EAFE0FF9094
:100C84006B80E0B50711C203906DA27403F01200EB
:100C940021755B01020DEF906EAC74FFF0020DEF55
:100CA400906EA4E0FF906BA3E06F6003020DEF90E1
:100CB4006EA4E004F0E4F55B906DA1F0020DEF305A
:100CC4000303020DEF906BA2E0D3940A5003020DCC
:100CD4006DA3E064026003020D6D906B6AE0FF9007
:100CE4006BACE06F6003020B10906B6BE0FF906BDA
:100CF400ADE06F6003020B10906B6CE0FF906BAE85
:100D0400E06F6003020B10906B6DE0FF906BAFE03F
:100D14006F6003020B10906B6EE0FF906BB0E06F9E
:100D24006003020B10906B6FE0FF906BB1E06F609B
:100D340003020B107E237F9812377F906BA463A26B
:100D440001906B6263A2017F12122C61906BB663F7
:100D5400A201906EAC63A2017F04122C61906DA27B
:100D64007406F0755B02020B107470446B7003021E
:100D74000B101245B3D203E4F55B906DA1F0906EB5
:100D8400B004F0E4906EA3F0A3F0200A5E7E237F0B
:100D9400A112377F8055300352906BA1E020E74BBE
:100DA400906BA3E0FF906EA3E0FE6F600D906EABBE
:100DB400E07007EE146F70338013906EA3E004F0BC
:100DC400906B5DE0FFD3940440031243C29068A982
:100DD4007482F0A37401F0906BA3E09068ABF07E92
:100DE400687FA97D03123FA6020B10200303020EA5
:100DF400AB9080D0E0700B906B75E0FEA3E0FF1227
:100E0400409AE55B7066906EB0E0D3943C403790B6
:100E14006EABE07031120006906EB07401F0E49095
:100E24006CA1F0A37412F0906EA4E0906CA3F0A3F4
:100E340074FDF09069B063A201906CA563A2017F78
:100E440012122C618006124429EF60207E6C7FA16F
:100E5400906CA2E02404FD123FA6906EABE0600308
:100E6400020B10906B81E0F55B020B10124590EFC2
:100E740060159068A97483F0E4A3F07E687FA97D6F
:100E840002123FA6020B10E55B64016003020B1023
:100E9400906DA1E004F0E0C3940540B0C203E4A364
:100EA400F0120021020B10E55B64016003020B10D9
:100EB400906DA2E0147003020F4F147003020F7BB5
:100EC4001470030210231470030210D924FE606905
:100ED40024066003020B10E4F55DF53C7459253CCF
:100EE400F582E4346AF583E0FF7462253CF582E41C
:100EF400346BF583EFF0053CE53CB43FDF200E2175
:100F0400906B7963A201906EAC63A2017F04122CF2
:100F140061906DA27401F0906DA1F0755B03020BFA
:100F240010906DA27404F0906DA17401F0755B14BF
:100F3400906EAC74FFF0020B10E4F55D12428690E3
:100F44006DA27401F0755B03020B10906EACE0604F
:100F54000B906B75E0FEA3E0FF12409A755B029064
:100F64006DA27402F0906B70E07003020B10906D30
:100F7400A27403F0020B10906EACE0700302101424
:100F8400906CA17480F0906CA37402F0E4A3F0A3BD
:100F940004F0906B6A63A201906CA663A2017F0ABD
:100FA400122C61906CB07430F0A3747BF0E4F53CC7
:100FB40074D8253CF582E43469F583E0FF6011744C
:100FC400B2253CF582E4346CF583EFF0053C80E017
:100FD40074B2253CF582E4346CF583747DF074B30B
:100FE400253CF582E4346CF583E4F0E53C2411906F
:100FF4006CA2F07C6E7DAC906B75E0FAA3E0FB7F95
:1010040002123EA17E6C7FA1E53C2413FD123FA693
:10101400906DA27404F0906B81E0F55B020B10906C
:101024006EACE070030210CA906CA17480F0906CF6
:10103400A37401F0E4A3F0A304F0A37430F0A37448
:101044007BF0E4F53C74D8253CF582E43469F583FF
:10105400E0FF601174A8253CF582E4346CF583EF5D
:10106400F0053C80E074A8253CF582E4346CF583FB
:10107400747DF074A9253CF582E4346CF583E4F0C6
:10108400E53C2407906CA2F07C6E7DAC906B75E01F
:10109400FAA3E0FB7F02123EA17E6C7FA1E53C2413
:1010A40009FD123FA6906EABE0601B1245B3D2035C
:1010B400E4F55B906DA1F0906EB004F0E4906EA343
:1010C400F0A3F0020B10906DA27404F0906B81E019
:1010D400F55B020B10906EACE0FF6009F4600690C3
:1010E40080027410F0200E2B755B02906DA1E064F9
:1010F40001FFF0A37401F0EF6005906B7980039019
:101104006B7D63A201906EAC63A2017F04122C611B
:10111400020B10755B14906EAC74FFF0020B108020
:01112400FECC
:0111250022A7
:10112600906BA2E0B444047F0180027F00906BA123
:10113600E0B447047E0180027E00EE5F604A906B59
:101146006AE0906BA3F0906B6BE0906BA4F0906BF1
:101156006CE0906BA5F0906B6DE0906BA6F0906BD9
:101166006EE0906BA7F0906B6FE0906BA8F0906BC1
:10117600A27452F0906B5763A2019080A863A201FB
:101186007F06122C61021634906B5DE0C394085002
:101196000302163D906B6AE0FF906BA3E06F60035D
:1011A60002163D906B6BE0FF906BA4E06F6003024C
:1011B600163D906B6CE0FF906BA5E06F6003021626
:1011C6003D906B6DE0FF906BA6E06F600302163DED
:1011D600906B6EE0FF906BA7E06F600302163D9088
:1011E6006B6FE0FF906BA8E06F600302163D906E98
:1011F600B5E060037401F0906EB67464F0906BA273
:101206007452F0906BA1E0644D703C7E237FAB126C
:10121600377F7E237FC112377F1245A47E237FE668
:1012260012377F7E237FF612377F7E247F021237A6
:101236007F7E247F0412377F7E247F0D12377F7EC8
:10124600247F0F12377F22906BA1E0644C70527E90
:10125600247F5C12377F906BA9E0F53DA3E0F53E55
:10126600E4F53F7D03AF3EAE3D1239437E247F97C2
:1012760012377FAE3DAF3EE4FB7D10123A217E244D
:101286007F0D12377F7410253EF53EE4353DF53D62
:10129600053FE53FC3941040CA7E247F0D12377F79
:1012A60022906BA1E0646C705CF5417E247F9A12FB
:1012B600377FE4F540AF417E007D031239437E243B
:1012C6007F9712377FE4F53FA841E6FF74AB253FD1
:1012D600F582E4346BF583EFF00541053FE53FB455
:1012E60010E67E6B7FABE4FB7D10123A217E247FF5
:1012F6000D12377F0540E540C3940840B87E247F31
:101306000D12377F22906BA1E0644B7046F53F7457
:1013160093253FF582E4346BF583E0FF601674A9EC
:10132600253FF582E4346BF583E0B50710053FE50C
:101336003FB408DB9069AD7432F0021634906BA1AD
:101346007421F0300A030216347E247FD512377FCB
:10135600021634906BA1E06452704E200A077E2478
:101366007FDD12377F906BAAE0906B5DF0E4F53F6E
:10137600906B5DE0FDE53FC39D5022906BA9E02593
:101386003F2458F582E4346AF583E0FF74AB253FC9
:10139600F582E4346BF583EFF0053F80D37E6B7FF7
:1013A600A1ED240AFD123E1B22906BA1E064497058
:1013B60045200A077E247FE812377F906BA9E0F567
:1013C6003DA3E0F53EE4F53F853E82853D83E0FFA3
:1013D60074AB253FF582E4346BF583EFF0053EE50B
:1013E6003E7002053D053FE53FB480DC7E6B7FA184
:1013F6007D8A123E1B22906BA1E0644460030214B6
:101406008D906BA9E0FF64447003021634EFB4318B
:101416000CC20A7E247FF012377F021634906BA925
:10142600E0B4300CD20A7E247FFC12377F021634D9
:10143600906BA9E0B4320CD20B7E257F0912377F60
:10144600021634906BA9E0B4330CC20B7E257F17CD
:1014560012377F021634906BA9E0B4340CD20C7E9E
:10146600257F2612377F021634906BA9E0B4350C1F
:10147600C20C7E257F3312377F021634906BA9E0AB
:10148600FF12001E0216349069ADE07013200A07A1
:101496007E257F4112377F906BA17421F0021634AE
:1014A6009069AD7432F0906BA1E0FFB45104C2AF05
:1014B60080FEEF64577045200A077E257F4F12375E
:1014C6007F906BAAE0906B5DF0E4F53F906B5DE07A
:1014D600FFE53FC39F400302163474AB253FF582F8
:1014E600E4346BF583E0FF906BA9E0253F2458F5C3
:1014F60082E4346AF583EFF0053F80D0906BA1E07B
:10150600645360030215AF200A077E257F5A1237FF
:101516007F906B6AE0FF906A61E06F703C906B6B46
:10152600E0FF906A62E06F7030906B6CE0FF906A4B
:1015360063E0B50724906B6DE0FF906A64E0B50741
:1015460018906B6EE0FF906A65E0B5070C906B6FC4
:10155600E0FF906A66E06F6016906BA17421F03030
:101566000A030216347E257F6912377F021634E499
:10157600F53FE4F55E7458253FF582E4346AF58359
:10158600E0FDAF3F124550053FE53FC394FE40E204
:10159600C2AFE4907FF0F0A3F0907FFD74AAF0A3B1
:1015A60074FFF0A37455F080FE906BA1E0644F7059
:1015B6004B906BA9E0F53DA3E0F53EE53E453D7059
:1015C6000A200A077E257F7212377F200A077F2AA4
:1015D6007E0012377FE4F53F74AB253FF582E43495
:1015E6006BF583E0853E82853D83F0053EE53E70E2
:1015F60002053D053FE53FB480DE8032906BA1E0F9
:10160600B4452B200A077E257F7912377F906BA978
:10161600E0FFA3E0907FF0CFF0A3EFF0C2AF907FA2
:10162600FD74AAF0A374FFF0A37455F080FE7E6BE0
:071636007FA17D08123E1B9D
:01163D00228A
:10438A00AE07EEC39430400BEED394395005EE24B9
:10439A00D0FF22EEC39461400BEED394665005EE33
:1043AA0024A9FF22EEC39441400BEED39446500554
:0843BA00EE24C9FF22AF062228
:1027D100C201E4906EB5F0D20EC204906EABF090DF
:1027E1006B6A63A201906EA563A2017F06122C6140
:1027F100E4F53DE53D75F003A424AAF582E4342512
:10280100F583E493FB740193FA740293F9121DE5C5
:1028110070030229B1E4F53EF53FFD74D82DF58230
:10282100E43469F583E0FF70030229ACE53D75F0FE
:1028310003A424AAF582E43425F583E493FB74010F
:1028410093FA740293F9853E82758300121DFEFE90
:10285100EFB50608753F01053E0229A8E53F700363
:102861000229A8EE60030229A3E53D24FE6022149B
:10287100700302299314700302299714700302292B
:102881009F240460030229AC906EB57401F0022903
:10289100ACD20174D82DF582E43469F583E0FF648C
:1028A1002D70030229AC12438AEFC454F0FC74D991
:1028B1002DF582E43469F583E0FF12438AEF2C9011
:1028C1006EA5F074DA2DF582E43469F583E0FF1228
:1028D100438AEFC454F0FC74DB2DF582E43469F5CE
:1028E10083E0FF12438AEF2C906EA6F074DC2DF585
:1028F10082E43469F583E0FF12438AEFC454F0FCAB
:1029010074DD2DF582E43469F583E0FF12438AEF2B
:102911002C906EA7F074DE2DF582E43469F583E026
:10292100FF12438AEFC454F0FC74DF2DF582E434C6
:1029310069F583E0FF12438AEF2C906EA8F074E0F2
:102941002DF582E43469F583E0FF12438AEFC45424
:10295100F0FC74E12DF582E43469F583E0FF124364
:102961008AEF2C906EA9F074E22DF582E43469F5BA
:1029710083E0FF12438AEFC454F0FC74E32DF58227
:10298100E43469F583E0FF12438AEF2C906EAAF0DC
:102991008019D2048015906EAB7401F0800DC20EC7
:1029A1008009E4F53FF53E0D02281C053D0227F4A0
:0129B1002203
:030003000241C9EE
:0D41C900C0E0C083C082C0D075D000C00728
:1041D600C2A8908008E0FFEF54F06035EF30E408A5
:1041E600D2079080087410F0EF30E508D20990806D
:1041F600087420F0EF30E608D2089080087440F08A
:10420600EF30E7069080087480F0908008E0FF8029
:09421600C690800874FFF0D2A8E4
:0B421F00D007D0D0D082D083D0E03296
:104286009080007480F0906B6263A201F583F582E2
:1042960063A2017F08122C61906B6A63A201908071
:1042A6008863A2017F0A122C61906B74E0FF9080F4
:1042B600B1F09080E1EFF09080957455F0A3F09006
:0C42C60080007401F09080097470F022F8
:043F2500AD07AC0632
:103F2900908009E04410F09080A0E0706F9080A12B
:103F39007482F09080A874FFF0A3F0A3F0A3F0AF0F
:103F490004AE079080AEEEF0AE05A3EEF0AE07909A
:103F590080ACEEF0AE05A3EEF09080007402F09014
:103F69006FD5121FD700000000906FD5E0908040F8
:103F7900F0906FD6E0908041F0906FD7E09080424A
:103F8900F0906FD8E0908043F0A3E4F0A3F0A3F0A1
:0C3F9900A3F0908018F0A3F0A3F0A3F0B8
:013FA50022F9
:04409A00AD07AC06BC
:10409E00908009E04440F09080D0E070559080D13F
:1040AE007482F0AF049080DEEFF0AF05A3EFF090D6
:1040BE0080027402F0906FD9121FD700000000909A
:1040CE006FD9E0908058F0906FDAE0908059F090C0
:1040DE006FDBE090805AF0906FDCE090805BF0A395
:1040EE00E4F0A3F0A3F0A3F0908030F0A3F0A3F0DF
:0240FE00A3F02D
:01410000229C
:103C5700908009E04420F09080B8E06003023CF8CF
:103C67009080B97482F07F039080C6EFF07FCDA378
:103C7700EFF07F039080C4EFF0A374CDF0301022F3
:103C8700906B79E09080C0F0906B7AE09080C1F003
:103C9700906B7BE09080C2F0906B7CE09080C3F0EB
:103CA700800C9080C074FFF0A3F0A3F0A3F0908085
:103CB700017402F0906FDD121FD700000000906FB3
:103CC700D9E090804CF0906FDAE090804DF0906FE3
:103CD700DBE090804EF0906FDCE090804FF0A3E443
:103CE700F0A3F0A3F0A3F0908024F0A3F0A3F0A337
:013CF700F0DC
:013CF80022A9
:103EA1008C3D8D3EA907EAFDE975F018A424ACFF0D
:103EB100E5F034808F82F583EDF0EBFDE975F018C4
:103EC100A4FFAEF024ACFBEE34808B82F583A3ED2E
:103ED100F0853E828C83E0FDEF24A8FFEE3480FE66
:103EE1008F82F583EDF0853E828C83A3E08F828EF5
:103EF10083A3F0853E82853D83A3A3E0FDE975F0B0
:103F010018A424A8FFE5F03480FE8F82F583A3A3D3
:103F1100EDF0853E828C83A3A3A3E08F828E83A3E1
:043F2100A3A3F02244
:063E1B008D42AB07AA0670
:103E2100906FD5E0FCA3E0FDA3E0FEA3E0F5468E94
:103E3100458D448C43AE02AF038E838F8263A20112
:103E4100E545540744C0F58385468263A201AF422C
:103E5100122CCA908000E020E5F9E4FCFDFEE54665
:103E61002542F546EE3545F545ED3544F544EC354D
:103E710043F543C2A8908040E543F0A3E544F0A395
:103E8100E545F0A3E546F0D2A89080007420F0AF9C
:0F3E910046AE45AD44AC43906FD5121FCBAF4248
:013EA00022FF
:063FA6008D3DAB07AA06E9
:103FAC00906FD9E0FCA3E0FDA3E0FEA3E0F5418E09
:103FBC00408D3F8C3EAE02AF038E838F8263A20195
:103FCC00E540540744D0F58385418263A201AF3D9F
:103FDC00122CCAE4FCFDFEE541253DF541EE3540D1
:103FEC00F540ED353FF53FEC353EF53EC2A89080EF
:103FFC0058E53EF0A3E53FF0A3E540F0A3E541F022
:10400C00D2A89080027420F0AF41AE40AD3FAC3EE0
:08401C00906FD9121FCBAF3DDC
:014024002279
:023BA9008F3E4D
:103BAB00908001E030E5037F0022906FDDE0FCA305
:103BBB00E0FDA3E0FEA3E0F5428E418D408C3F90EB
:103BCB006EA563A201E541540744C8F58385428283
:103BDB0063A2017F06122CE0E5422406F542E43590
:103BEB0041F541E43540F540E4353FF53F906DA399
:103BFB0063A201E541540744C8F58385428263A261
:103C0B0001AF3E122CE0E4FCFDFEE542253EF54201
:103C1B00EE3541F541ED3540F540EC353FF53FC212
:103C2B00A890804CE53FF0A3E540F0A3E541F0A35D
:103C3B00E542F0D2A89080017420F0AF42AE41ADC6
:0B3C4B0040AC3F906FDD121FCBAF3E7E
:013C5600224B
:10367300C2A89081E0E0F53D053D053D053D053DD2
:10368300053D053D053D053D053D053D908010E0AB
:10369300F540A3E0F541A3E0F542A3E0F5439081B3
:1036A300E1E0F53D053D053D053D053D053D053D98
:1036B300053D053D053D053D908014E0F544A3E03F
:1036C300F545A3E0F546A3E0F547D2A8E546B542A4
:1036D30008E547B543037F0022E4F53DE54654077B
:1036E30044E0F58385478263A201906BA163A20145
:1036F3007F08122CF8906BA363A201906B5763A20F
:10370300017F06122C61906BA1E0F53EA3E0F53F2B
:10371300E4F53D906BA1E0702AA3E024F8F53DE5C4
:1037230046540744E0F58385478274082582F58271
:10373300E43583F58363A201906BA163A201AF3DDE
:10374300122CF8AE3EE4FCFDE547253FF547E54680
:103753003EF546ED3545F545EC3544F544C2A890B4
:103763008014E544F0A3E545F0A3E546F0A3E5475F
:0B377300F0D2A89080007440F0AF3D41
:01377E002228
:102EDC00C2A89081E6E0F53D053D053D053D053D6B
:102EEC00053D053D053D053D053D053D908028E032
:102EFC00F540A3E0F541A3E0F542A3E0F543908152
:102F0C00E7E0F53D053D053D053D053D053D053D30
:102F1C00053D053D053D053D90802CE0F544A3E0C5
:102F2C00F545A3E0F546A3E0F547D2A8E4F53DE569
:102F3C0046B5420AE547B54305C20802303AE546B4
:102F4C00540744F0F58385478263A201906BA1631B
:102F5C00A2017F08122CF8906BA1E0F53EA3E0F5DE
:102F6C003FE53F453E70099080027410F07F0022CF
:102F7C00906EACE0FFF4602D906BA3E06F707690D8
:102F8C006EADE0FF906BA4E06F706A906EAEE0FFE8
:102F9C00906BA5E06F705E906EAFE0FF906BA6E05B
:102FAC006F60228050906BA3E0906EACF0906BA49D
:102FBC00E0906EADF0906BA5E0906EAEF0906BA6CD
:102FCC00E0906EAFF0906BA1E0702AA3E024F8F5CE
:102FDC003DE546540744F0F5838547827408258205
:102FEC00F582E43583F58363A201906BA163A201A2
:102FFC00AF3D122CF8AE3EE4FCFDE547253FF5470E
:10300C00E5463EF546ED3545F545EC3544F544AF22
:10301C0043AE42AD41AC40AB47AA46A945A844D308
:10302C00121F9A40099080027410F07F0022C2A8EF
:10303C0090802CE544F0A3E545F0A3E546F0A3E52C
:0C304C0047F0D2A89080027440F0AF3D25
:013058002255
:10305900C2A89081E3E0F53D053D053D053D053DEF
:10306900053D053D053D053D053D053D90801CE0BF
:10307900F540A3E0F541A3E0F542A3E0F5439081D3
:10308900E4E0F53D053D053D053D053D053D053DB5
:10309900053D053D053D053D908020E0F544A3E053
:1030A900F545A3E0F546A3E0F547D2A8E4F53DE5EB
:1030B90046B5420AE547B54305C2090231A1E546CD
:1030C900540744E8F58385478263A2019068AD639C
:1030D900A2017F0E122D0E9068ADE0F53EA3E0F53A
:1030E9003F906EA5E0FF9068B5E06F706C906EA69A
:1030F900E0FF9068B6E06F7060906EA7E0FF90689F
:10310900B7E06F7054906EA8E0FF9068B8E06F70F8
:1031190048906EA9E0FF9068B9E06F703C906EAA84
:10312900E0FF9068BAE06F70309068ADE0702AA354
:10313900E024F2F53DE546540744E8F583854782E6
:10314900740E2582F582E43583F58363A2019068C4
:10315900AD63A201AF3D122D0EAE3EE4FCFDE54785
:10316900253FF547E5463EF546ED3545F545EC3550
:1031790044F544AF43AE42AD41AC40AB47AA46A982
:1031890045A844D3121F9A5006E53F453E70099061
:1031990080017410F07F0022C2A8908020E544F0DD
:1031A900A3E545F0A3E546F0A3E547F0D2A8908052
:0631B900017440F0AF3D7F
:0131BF0022ED
:04377F008E428F43A4
:10378300906FD5E0FCA3E0FDA3E0FEA3E0F5498E36
:10379300488D478C46E549FFE5485407FEE42FF57D
:1037A30045EE34C0F544854582F5837423F0054521
:1037B300E545700205445344C7F582854483740A82
:1037C300F00545E545700205445344C7906B6A63B1
:1037D300A20185448385458263A2017F06122CCA18
:1037E30074062545F545E43544F544854283854310
:1037F3008263A20185448385458263A201122CAEB4
:10380300908000E020E5F9E4FCFDFE906FD5E0F840
:10381300A3E0F9A3E0FAA3E02FFFEE3AFEED39FDB2
:10382300EC38FCEF2408FFE43EFEE43DFDE43CFC01
:10383300906FD5121FCBC2A8906FD5E0908040F057
:10384300906FD6E0908041F0906FD7E0908042F087
:10385300906FD8E0908043F0D2A89080007420F05D
:013863002242
:063A21008E428F438D442C
:103A2700906FD5E0FCA3E0FDA3E0FEA3E0F54A8E8E
:103A3700498D488C47E54AFFE5495407FEE42FF5D1
:103A470046EE34C0F545854682F5837423F0054676
:103A5700E546700205455345C7F582854583EBF07A
:103A67000546E546700205455345C7906B6A63A254
:103A77000185458385468263A2017F06122CCA749D
:103A8700062546F546E43545F54585428385438257
:103A970063A20185458385468263A201AF44122C48
:103AA700CA908000E020E5F974082544F544FFE456
:103AB700FCFDFEE54A2FF54AEE3549F549ED354857
:103AC700F548EC3547F547C2A8908040E547F0A395
:103AD700E548F0A3E549F0A3E54AF0D2A8908000B5
:103AE7007420F0AF4AAE49AD48AC47906FD5121F6E
:013AF700CB03
:013AF80022AB
:063943008E428F43AB052C
:10394900906FD5E0FCA3E0FDA3E0FEA3E0F5498E6E
:10395900488D478C46E549FFE5485407FEE42FF5B5
:1039690045EE34C0F544854582F5837423F0054559
:10397900E545700205445344C7F582854483EBF05D
:103989000545E54570020544906B6A63A2018544CB
:103999008385458263A2017F06122CCA74062545D8
:1039A900F545E43544F5445344C7E54285458285E8
:1039B9004483F00545E545700205445344C7F58243
:1039C900854483E543F00545E545700205445344C4
:1039D900C7908000E020E5F9E549240AF549E43576
:1039E90048F548E43547F547E43546F546C2A89019
:1039F9008040E546F0A3E547F0A3E548F0A3E54993
:103A0900F0D2A89080007420F0AF49AE48AD47AC21
:073A190046906FD5121FCB90
:013A20002283
:1044FA00E5D220E0FBC2AF438E2075D2028F8275CF
:0C450A008300E0FFE4F5D2538EDFD2AF57
:014516002282
:10455000E5D220E0FBC2AF43D2028F82758300ED2B
:0A456000F075D25063D250D2AF22A2
:10402500E4FEEE04FF1244FA74622EF582E4346B6A
:10403500F583EFF00EBE3FEAE4FEEE247FFF124467
:10404500FA74D82EF582E43469F583EFF074D82E2E
:10405500F582E43469F583E0701B74D82EF582E4AB
:104065003469F5837420F074D92EF582E43469F54A
:1040750083E4F080040EBE80C1E4906A57F0FEAF81
:10408500061244FA74582EF582E4346AF583EFF08B
:044095000EBEFEEB72
:014099002204
:10451700A2AF9223C2AF8C838D82EF122D2643A2C6
:0C45270020122D2853A2DFA22392AFFF28
:014533002265
:02448E008F3D60
:10449000A2AF9223C2AFE4F5838D827406122D265B
:1044A000E53D43A220122D2853A2DFA22392AF7F25
:0144B000010A
:0144B10022E8
:0244B2008F3D3C
:1044B400A2AF9223C2AFE4F5838D82740A122D2633
:1044C400E53D43A220122D2853A2DFA22392AF7F01
:0144D40001E6
:0144D50022C4
:102B8600A907E7FFA805EF93C3966008403B74FCCE
:102B96002FFF80F00F08EF93C3966008402B74FB5D
:102BA6002FFF80E00F08EF93C3966008401B74FA6E
:102BB6002FFF80D00F08EF93D3966008400B74F96F
:102BC6002FFF80C01F1F1F1F1FEF54FEF80303F7C0
:102BD600E893FC08E893FD08E893FE08E893FF22D3
:102BE60009E993C39D6008402974FB29F980F1091E
:102BF600E993C39E6008401A74FA29F980E209E94C
:102C060093D39F6008400B74F929F980D3191919D9
:102C16001919E9C313C313FF22740093F8ECC39880
:102C26004024701F740193F8EDC398401970147412
:0E2C36000293F8EEC398400E7009740393F8F1
:102C4400EFC39840037F00227F0122EDF8E6F008ED
:102C5400A3DFFA22EDF8E0F608A3DFFA22E0A3638B
:102C6400A201F0A363A201DFF475A20022E0A36332
:102C7400A201F0A363A201E0A363A201F0A363A2F3
:102C840001E463A201F0A363A201DFE175A20022C3
:102C9400E0A363A2016DFE936CFDEE058393FC1526
:102CA4008363A201DFEA75A200227F00E493A36399
:102CB400A201F00F600CA3E583C2E3F58363A201D4
:102CC40080EA75A20022E0A363A201F0A3E583C217
:102CD400E3F58363A201DFEE75A20022E0A363A201
:102CE40001F0A3E583C2E4D2E3F58363A201DFEC40
:102CF40075A20022E583C2E3F583E0A363A201F099
:102D0400A363A201DFEE75A20022E583C2E4D2E34D
:102D1400F583E0A363A201F0A363A201DFEC75A233
:102D24000022F922C002C004C00612FFF0D006D06F
:042D340004D00222A3
:1042D20020536572763A0020547261737353656E8F
:1042E200644552520A00205265496E697420434166
:1042F2004E0A002043414E283029203E20544F21AF
:104302000A0020545520300A0020545520310A005A
:03001E00E4FF22DA
:10445C00C28DC2AF438901C28C906ECBE0FF700756
:10446C00F58A758CEE8016EFB40508E4F58A758C28
:10447C00B8800AEFB40A06E4F58A758C70D28CD237
:02448C00AF225D
:10431200C28DC2AF438901C28C906ECBE0FF701494
:10432200302209F58A758CDCC222801E758A667578
:104332008CFC8016EFB40508E4F58A758CEE800AD1
:0F434200EFB40A06E4F58A758CDCD28CD2AF2278
:10453400124101120022D221E4F537906FD3F0F535
:0C45440025F53B12445CC222E4F539224C
:1043C200EF24FCF53D200A127E427FD212377F7E17
:1043D2006B7FA57B01AD3D123A21906BA563A201D3
:1043E200906F5363A201AF3D122C61853D25E4F528
:0343F20036C21FB1
:0143F50022A5
:0F458100D3EF6480948E5006E53B70028F3B228F
:1025BF00208D0302265BC28C2021030226B4E52561
:1025CF00605474572536F582E4346FF583E02405A3
:1025DF00F53DD3940E4008E4F525D21F0226B474BE
:1025EF00532536F582E4346FF5837D27AF3D122CEA
:1025FF0058E53D2536F536E52730E702D22212445D
:10260F005C12422AE536C3952550030226B4E4F541
:10261F0025D21F0226B4E5386014906EB77D27FFD0
:10262F00122C5812445C12422AE4F5388077E53BAD
:10263F0060149068AD7D27FF122C5812445C124233
:10264F002AE4F53B805F12416612445C1232F58F2B
:10265F003DEF6051124312E4F539E53AC3946E50E1
:10266F001874CC253AF582E4346EF583E53D253AAE
:10267F00F53A7D27AF3D122C4F300124E52730E787
:10268F000330101C906DA37D27AF3D122C4FAF3D33
:10269F00123BA9EF700A200A077E427FD912377FBB
:1026AF00AF3D1220CD300D1E906610E0C394FA504E
:1026BF0003E004F030000D0539E539D394F0400400
:1026CF00C2AF80FEC20D2002030227CDE537603175
:1026DF00D39401400415378028906FD3E004F0E0C5
:1026EF00D39403400D200A077E427FE812377F12F2
:1026FF004534200A077E427FF512377FE4F537D243
:10270F0021302043E538703F906EB704F0A3740872
:10271F00F0A37480F0A37401F0A37406F0906F4ED1
:10272F00E0906EBCF0906F4FE0906EBDF0906F50E8
:10273F00E0906EBEF0906F51E0906EBFF0E4A3F0AA
:10274F00A3F075380BC220301E72906F4CE07035BD
:10275F00E5387031906EB77442F0A37408F0906F43
:10276F004DE0906EB9F0906F52E0906EBAF0A37496
:10277F0001F0753806200A077E437F0412377F90D9
:10278F006F4CE004F0906F4CE06402702FE53870EE
:10279F002B906EB77402F0A37408F0906F4DE09019
:1027AF006EB9F0A3F0A37401F0753806200A077E06
:1027BF00437F0B12377F906F4CE004F0C202120080
:0127CF0026E3
:0127D00022E6
:10442900E53A602CE4906CA1F0A3E53AF0906EA413
:10443900E0906CA3F0A37419F0906ECC63A2019084
:104449006CA563A201AF3A122C61E4F53A7F01220F
:034459007F0022BF
:0B459000301F05C21F7F01227F0022A8
:0100210022BC
:0645B300E4F53AF52522B3
:100006007F01E49069B0F0A3F0A3F0FEEF25E0FFD6
:040016000EBE08F81A
:01001A0022C3
:1044D6002043616E457247495400200A002043611B
:1044E6006E457272434821000A000A2052657145E2
:0444F60072722100BD
:1032F500E59B541F6020200A1A7E447FD612377F33
:10330500E59B541FFF7E007D031239437E447FE019
:1033150012377FE4F59BE5BA30E010E4F5B375B1FB
:1033250080F5B2D221F537906FD3F0E5CFF4700375
:10333500023424753F01E4F53EE5CFF4553F7003B3
:10334500023412E53EC454F0F5B1E5B2547F642071
:1033550060030233E3E5B3540FF52B85BC2720103A
:1033650016E5BD541FFF131313541FFFE5BD54E0AD
:1033750044184FF5288006E5BD54E0F528E5BDC4A1
:103385003354E0FFE5BE131313541F4FF529E5BE73
:10339500C43354E0FFE5BF131313541F4FF52A85BB
:1033A500A32C85A32D85A32E85A32F85A33085A3C7
:1033B5003185A33285A333E4F5B230100C85AE34E4
:1033C50085AF3575B3D07F0F22E527547EB5270528
:1033D50075B350800375B3D0E52B2405FF22E5B204
:1033E500549F6023200A207E447FE312377FAFB2CB
:1033F5007E007D03123943AFB37E007D031239434E
:103405007E447FEE12377FE4F5B275B3D0E53F25F4
:10341500E0F53F053EE53EC39408500302333E7F89
:0134250000A6
:013426002283
:10422A0020105875B180E4F5B3F5B28527BCE529AD
:10423A00C4135407FFE52854E04FF5BDE52933338D
:10424A003354F8FFE52AC41354074FF5BEE52A3361
:10425A00333354F8F5BF852CA3852DA3852EA3856A
:10426A002FA38530A38531A38532A38533A3E52BFC
:0C427A00540F2450F5B375370AC22122FE
:1041660020105F75B190E5B220E613200A107E4458
:104176007FF012377FAFB27E007D03123943E4F53C
:10418600B3F5B274862516F582E43461F583E0F55D
:10419600BCE4F5BD74872516F582E43461F583E049
:1041A600FF33333354F8F5BE75BF7805160516741C
:1041B600862516F582E43461F583E07002F51675FE
:0341C600B35022D1
:09459B00EF6003C29622D29622C1
:1041010043AB01C2E8C2EAE4FFEFC454F0F5B1C326
:10411100EF64809488500575B3D08003E4F5B3E46F
:10412100F5B2F5BCF5BDF5BEF5BFF5C4F5C5F5C6EF
:10413100F5C7F5A3F5A3F5A3F5A3F5A3F5A3F5A39A
:10414100F5A30FBF0EC3906ECBE0FF25E0F5B4756C
:10415100B50C75B66C75A11275AB0275C13E75C310
:04416100FF75C20321
:014165002237
:1029B2000000000000000000000000000000000015
:1029C2003FF3630041D5E80043B71B8045984F00B1
:1029D20047798280495C07804B3D3B004D1E6E80EB
:1029E2004EFFA20050E2270052C35A8054A48E0028
:1029F2005685C180586846805A497A005C2AAD8063
:102A02005E0BE1005FEE660061CF998063B0CD009E
:102A120065920080677485806955B9006B36EC80D9
:102A22006D1820006EFAA50070DBD880000000004F
:102A32000028DE80004DC8800076A700009E34008A
:102A420000C7123000EE9F8001177E0001405C80BB
:102A52000167E9800190C80001B8550001E13380A7
:102A6200000000000028DE80004F1A000077F88086
:102A7200009F858000C8640000EFF1000118CF803C
:102A82000141AE0001693B000192198001B9A680A3
:102A920001E2850000000000000151800002A30055
:102AA2000003F48000054600000697800007E90055
:102AB20000093A80000A8C00000BDD80000D2F0017
:102AC200000E8080000FD2000011238000127500DA
:102AD2000013C68000151800001669800017BB009D
:102AE20000190C80001A5E00001BAF80001D01005F
:102AF200001E5280001FA4000020F5800022470023
:102B0200002398800024EA0000263B8000278D00E5
:102B12000028DE800000000000000E1000001C20D3
:102B220000002A3000003840000046500000546087
:102B3200000062700000708000007E9000008CA097
:102B420000009AB00000A8C00000B6D00000C4E0A7
:102B52000000D2F00000E1000000EF100000FD20B4
:102B620000010B30000119400001275000013560BF
:102B720000014370000151801F1C1F1E1F1E1F1FDA
:042B82001E1F1E1FD5
:10355000E54F25E025E024B2F582E43429F5831215
:103560001FAB8F588E578D568C55E54F54037028DE
:10357000E55425E025E0245EF582E4342AF5831243
:103580001FABEF2558F558EE3557F557ED3556F585
:1035900056EC3555F5558026E55425E025E0242ADE
:1035A000F582E4342AF583121FABEF2558F558EE67
:1035B0003557F557ED3556F556EC3555F555E5517A
:1035C00025E025E02492F582E4342AF583121FAB2E
:1035D000EF2558F558EE3557F557ED3556F556ECBD
:1035E0003555F555E552C3940C402AE55824C0F5ED
:1035F00058E55734A8F557E43556F556E43555F5F2
:1036000055E55224F4FF7E007C0E7D10121E2BAA7D
:1036100006AB07800FAF527E007C0E7D10121E2B72
:10362000AA06AB07AE02E4FCFDE5582BF558E557BA
:103630003EF557ED3556F556EC3555F555E55375D0
:10364000F03CA4FFAEF0E4E5582FF558E5573EF501
:1036500057ED3556F556EC3555F555E4FEE558254C
:1036600050F558EE3557F557ED3556F556EC3555BE
:02367000F5550E
:013672002235
:1031C000906FEBE0F54F25E025E024B2F582E43482
:1031D00029F583E54FD3941F501DAF58AE57AD5618
:1031E000AC55122C1FEF700F74042582F582E43564
:1031F00083F583054F80DC74FC2582F58274FF35EE
:1032000083F583AF82121FBBC3E5589BF558E55782
:103210009AF557E55699F556E55598F555154FE544
:103220004F14906FEBF0E54F54037005902A6280C5
:1032300003902A2E7554307F547D55122B86A80496
:10324000A905AA06C3E5589FF558E5579AF557E52D
:103250005699F556E55598F5550554902A96AF5868
:10326000AE57AD56AC557B007A00797C122BE68FB9
:1032700051EF25E025E02496F582E4342AF5831207
:103280001FBBC3E5589BF558E5579AF557E5569986
:10329000F556E55598F5550551902B16AF58AE5794
:1032A000AD56AC557B007A00795C122BE68F52EF5D
:1032B00025E025E02416F582E4342BF583121FBBAC
:1032C000C3E5589BF558E5579AF557E55699F556D5
:1032D000E55598F555AE57AF587C007D3C121E3D24
:1032E0008D50AE57AF587C007D3C121E3D8E578FDF
:0532F00058855853222F
:101A4B0042415544004D41584200525453004445C5
:101A5B004C4159005452414E5A0043414E004B5099
:101A6B0000544F52455000002D2D2D2D2D20CFE031
:101A7B00F0E0ECE5F2F0FB20495020EFF0EEF2EE57
:101A8B00EAEEEBE0202D2D2D2D2D2D2D2D2D2D2D99
:101A9B002D4C494E4B434F4E54522C2CCFE5F0E579
:101AAB00E7E0E3F0F3E7EAE020EFF0E820EEF2F115
:101ABB00F3F2F1F2E2E8E820F1EEE5E4E8EDE5ED32
:101ACB00E8FF20F120F1E5F0E2E5F0EEEC2C4C2CF8
:101ADB00CDE5F23D2CC4E03D4C494E4B434F4E54AB
:101AEB00520054524153532C2CCCEEF1F2EEE2EE59
:101AFB00E920EAEEEDF2F0EEEBEBE5F02C4C2CCD21
:101B0B00E5F23D2CC5F1F2FC3D54524153532D00EF
:101B1B004E4F4C494E4B2C2CD1E2FFE7FC20F120D1
:101B2B00F1E5F0E2E5F0EEEC20EFEE2049502C4C25
:101B3B002CCDE5F23D4E4F4C494E4B2CC5F1F2FCF2
:101B4B003D2D2D2D2D2D20CFE0F0E0ECE5F2F0FB1F
:101B5B0020F4F3EDEAF6E8EEEDE0EBFCEDFBF5201F
:101B6B00E1EBEEEAEEE2202D2D2D2D2D2D2D2D2D41
:101B7B002D2D2D4D4158422C4D4158423232322C95
:101B8B00CAEEEBE8F7E5F1F2E2EE20E1EBEEEAEE7E
:101B9B00E220D2D120D2C8D220D2D32C44332C3045
:101BAB002D380043414E2C43414E302C43EAEEF08E
:101BBB00EEF1F2FC20F8E8EDFB2043414E2C4C2CCF
:101BCB00353030EAE13D2C3530EAE13D43414E35CD
:101BDB00002D2D2D2D2D20CFE0F0E0ECE5F2F0FBCC
:101BEB0020EFF0EEF2EEEAEEEBE020CCDDCA20388F
:101BFB0037302D352D313031202D2D2D2D2D2D2DF7
:101C0B002D2D2D2D2D424155442C42415544313221
:101C1B0030302CD1EAEEF0EEF1F2FC20EEE1ECE507
:101C2B00EDE02C4C2C3130302C3230302C3330302A
:101C3B002C3630302C313230302C323430302C3496
:101C4B003830302C393630302C31393230302C336F
:101C5B00383430302C35373630302C31313532305A
:101C6B0030004B502C4B50312CCDEEECE5F020CA14
:101C7B00CF28525455292C44312C312D3235350077
:101C8B00005265737461727420424C0A0043414EDA
:101C9B00205455204F4B0A0043414E20545520529F
:101CAB0065710A002054552054696D654F555421B8
:101CBB000A00204F4B2000204E414B200020526544
:101CCB00732043480A2000205265732055500A2088
:101CDB00002044415441410A200020545553656C67
:101CEB000A2000205455455845430A200020444102
:101CFB0054410A20002053657454696D650A200015
:101D0B00204348520A2000205245510A20002054FB
:101D1B00555F4F4B0A20002054555F4572720A20C5
:101D2B000020545552656164790A200020545552A5
:101D3B0065616479320A200073656E642074730ADE
:101D4B000073656E642074734379630A00207365B6
:101D5B006E64207469744379630A20002073656E86
:101D6B0064207469690A20002073656E64207469AD
:101D7B007453706F740A2000C7E0E3F0F3E7EEF7DB
:101D8B00EDFBE920EEE1F0E0E73A20CACF20C8F105
:101D9B00E5F2FC28CCDDCA3837302D352D3130310A
:101DAB0029207620312E30310A00FF1A4BFF1A50B2
:101DBB00FF1A55FF1A59FF1A5FFF1A65FF1A69FFC1
:101DCB001A6CFF1A72FF1A73FF1AEDFF1B1BFF1B16
:0A1DDB00AEFF1BDCFF1C6DFF1C8B2C
:030023000234277D
:0B342700C0E0C083C082C0D075D01888
:1034320020980302350EC298755C01AF99301303D0
:10344200023547D29120113CBFE507D21DD21302AB
:10345200350EBFA207D216D21302350EBF680DD2A7
:1034620011D218750A00750E0002350EEF64106055
:103472000302350ED211D219751502750E03750AA3
:1034820000023547E50E70078F15050E023547E538
:103492000EB4010FE515B51F05050E023547C21121
:1034A200023547E50EB4020AEF646860CEC211022B
:1034B2003547E50EB4031E7467250FF582E43466C2
:1034C200F583EFF0050F250AF50A1515E515707558
:1034D200750E048070E50EB4040DE50AB51F0405EF
:1034E2000E8062C211805EE50E6405701FBF161168
:1034F200D213850F15630F80530F80C211C29180C2
:1035020044C219C218530F80C21180393099363023
:103512001231906185E0FFE510C39F4008C212D2CC
:103522001AC290801ED29074A72510F582E43467E7
:10353200F583E0F513E50B5213A2D0B3929B8513EA
:05354200990510C2997B
:09354700D0D0D082D083D0E03254
:10163E00E4906407F0906ECBF0906406F0906FE942
:10164E007461F0A37486F0906FE9E475F001121ED8
:10165E009285F082F58374C4F0906FE9E475F00121
:10166E00121E9285F082F583E4F0906FE975F00119
:10167E00121E9285F082F58374C4F0906FE9E475C2
:10168E00F001121E9285F082F5837401F0906FE9DD
:10169E00E475F001121E9285F082F58374C8F09005
:1016AE006FE9E475F001121E9285F082F583E4F085
:1016BE00906FE975F001121E9285F082F58374C861
:1016CE00F0906FE9E475F001121E9285F082F583B9
:1016DE007401F0906FE9E475F001121E9285F082AC
:1016EE00F58374C2F0906FE9E475F001121E9285D5
:1016FE00F082F583E4F0906FE975F001121E928589
:10170E00F082F58374C2F0906FE9E475F001121E59
:10171E009285F082F5837401F0906FE9E475F00123
:10172E00121E9285F082F583E4F0906FE975F00158
:10173E00121E9285F082F583E4F0F516906FE1F0BB
:10174E00906FE1E075F003A424B5F582E4341DF545
:10175E0083E493FB740193FA740293F9121DE570FE
:10176E0003021A4AE4906FE3F0A3F0906FE2F09058
:10177E006FE2E024D8F582E43469F583E0FF70036C
:10178E00021A41906FE1E075F003A424B5F582E4EE
:10179E00341DF583E493FB740193FA740293F9906C
:1017AE006FE3E0F582758300121DFEFEEFB5060FA6
:1017BE00906FE47401F0906FE3E004F0021A389039
:1017CE006FE4E07003021A38EE6003021A2F906F76
:1017DE00E1E0B408004003021A419017EFF8282800
:1017EE007302180702185402196B021970021807B7
:1017FE0002199F0219CF0219FF906FE2E024D8F967
:10180E00E43469FA7B01C0031B8B407541007542BD
:10181E0000E4F543D003122D38906FE5121FCB90E4
:10182E006FE5E0F8A3E0F9A3E0FAA3E0FB7F007E0A
:10183E008C7D0A7C00121EE4121F769068A7EEF0D3
:10184E00A3EFF0021A41906FE97461F0A37486F071
:10185E00906FE2E024D8F582E43469F583E024D079
:10186E00F516C394014007E516D394084003E4F53A
:10187E0016E5166028906FE9E475F001121E928548
:10188E00F082F58374C4F01516906FE9E475F001DB
:10189E00121E9285F082F583E516F080D4906FE2E9
:1018AE00E024D9F582E43469F583E024D0F516C33B
:1018BE0094014007E516D394084003E4F516E516A7
:1018CE006028906FE9E475F001121E9285F082F5A2
:1018DE008374C8F01516906FE9E475F001121E922C
:1018EE0085F082F583E516F080D4906FE2E024DA7D
:1018FE00F582E43469F583E024D0F516C3940140F3
:10190E0007E516D394084003E4F516E51660289013
:10191E006FE9E475F001121E9285F082F58374C2B0
:10192E00F01516906FE9E475F001121E9285F082A3
:10193E00F583E516F080D4906FE9E475F001121E80
:10194E009285F082F583E4F0906FE975F001121E36
:10195E009285F082F583E4F0F516021A41D2170251
:10196E001A41906FE2E024D8F9E43469FA7B01C0A1
:10197E00031B8B40754100754200E4F543D0031202
:10198E002D38906FE5121FCB906FE8E0F509021A23
:10199E0041906FE2E024D8F9E43469FA7B01C00388
:1019AE001B8B40754100754200E4F543D003122DA8
:1019BE0038906FE5121FCB906FE8E0906ECBF08001
:1019CE0072906FE2E024D8F9E43469FA7B01C00327
:1019DE001B8B40754100754200E4F543D003122D78
:1019EE0038906FE5121FCB906FE8E0906407F0809F
:1019FE0042906FE2E024D8F9E43469FA7B01C00327
:101A0E001B8B40754100754200E4F543D003122D47
:101A1E0038906FE5121FCB906FE8E0906406F0806F
:101A2E0012E4906FE4F0906FE3F0906FE2E004F058
:0C1A3E0002177D906FE1E004F002174EEB
:011A4A002279
:103864009069AEE064557004A3E064816064E4F59B
:103874001074112510F582E43466F583E4F07408BD
:103884002510F582E43466F583E4F074FE2510F522
:1038940082E43462F583E4F00510E510B408D2E460
:1038A400F51074672510F582E43467F583E4F005B8
:1038B40010E510B440ECE4F51074B62510F582E47C
:1038C4003461F583E4F00510E510B480ECE4F512FE
:1038D400F511E4906FEBF0C212C21AC211C213F5D3
:1038E40010906185F0F509F508F50FF55CC20FC27B
:1038F4001CC2179068A774FFF0A374F4F0750BFF53
:1039040012163EC291C290C2ADE4F5C9D2CDD2CC5A
:10391400C2C9C2CAF5CDF5CC9068A7E0F5CBA3E047
:10392400F5CA85CBCD85CACCD29FD29ED29CD2CAB1
:0F393400C2ACC298C29975B81075B710D2AC2248
:023AF9008F41FB
:103AFB00E4FF7C617D00FEEEC3954150120DEDAAF3
:103B0B000470010C14F5828A83E02FFF0E80E80D00
:103B1B00EDAA0470010C14F5828A83EFF00DEDAE63
:103B2B000470010C14F5828E837416F00541054167
:103B3B007E677FA77C617D00E541B4040E8F828E8A
:103B4B00837410F00FBF00010E80328F828E83744E
:103B5B0068F00FBF00010EE54124FEFB8F828E83C0
:103B6B00F00FBF00010E8F828E83EBF00FBF0001B1
:103B7B000E8F828E837468F00FBF00010E8C838DC5
:103B8B008263A2018E838F8263A201AF41122C61EB
:0D3B9B00E541B4040304FF22E5412404FFCA
:013BA80022FA
:10435100201235123AF9906185EFF0200A0B7E6741
:104361007FA7E0FDE4FB123A213017057F011245DA
:104371009BE5096003F55922E4906610F0F510D22F
:0943810012C2992099FDD2992283
:0220CD008F3E44
:1020CF00906407E07003022380E52730E712E52ACA
:1020DF00B4100D200A077E1C7F8C12377FE4F508A1
:1020EF00E52724BE700302234D24FA7003022275E4
:1020FF0024046003022380E52830E70302219EE5D4
:10210F002A6066E529C394024003022380E5297003
:10211F0007E52A14F53F8006E52A241FF53FE53F22
:10212F0075F004A42406F582746335F0F5837D2CD5
:10213F007F04122C4FE53F75F004A424FEF5827442
:10214F006135F0F5837D307F04122C4F74F625290D
:10215F00F582E43461F5837481F074B6253FF5821E
:10216F00E43461F5837401F02274082529F582E4C3
:10217F003466F583E04480F0E52925E025E0243B33
:10218F00F582E43466F5837D2C7F04122C4F22E513
:10219F002B64086003022380753E01E52A5407FF74
:1021AF00E53EA807088002C333D8FCF53E74082526
:1021BF0012F512B5110674082511F511E52A547F91
:1021CF00FFE529C43354E02FFE74002512F582E495
:1021DF003460F583EEF0E52AC39480503CEF13137F
:1021EF0013541FFFE52925E025E025E025E0243BDA
:1021FF00F582E43466F583E5822FF582E43583F5C5
:10220F0083E0FFE53EF4FEEF5EF074012512F582E8
:10221F00E43460F583E4F0803AE52A547FFF13132A
:10222F0013541FFFE52925E025E025E025E0243B99
:10223F00F582E43466F583E5822FF582E43583F584
:10224F0083E0453EF074012512F582E43460F58396
:10225F007401F074022512F582E43460F5837D2C4D
:10226F007F06122C4F22E52A54E06440702CE52A99
:10227F00540F144440FF74FE2529F582E43462F5AF
:10228F0083EFF0E52925E025E0241AF582E4346692
:10229F00F5837D2C7F04122C4F2274FE2529F582A5
:1022AF00E43462F583E0F55330E64AE52A1313541C
:1022BF003FFFE553540FB50714E55354074480FF10
:1022CF0074FE2529F582E43462F583EFF0E52A5494
:1022DF007FFF1313543FFF75F008E529A42FF582F4
:1022EF00E435F0F583E5822467F582E5833467F5FD
:1022FF0083E4F08027E52A547FFF1313543FFF75C3
:10230F00F008E529A42FF582E435F0F583E5822462
:10231F0067F582E5833467F5837401F075F040E566
:10232F0029A42408F582E5F03464F583E52A547F67
:10233F0075F0021220087D2CAF2B122C4F22301E6D
:10234F0030E52AB40112200A077E1C7F9812377FCE
:10235F00E52D04906FD4F022E52AB40314906F4C4E
:10236F00E0B401037405F0200A077E1C7FA3123727
:01237F007FDE
:01238000223A
:1000260030001DC200301E18906182E004F0E0D35B
:100036009414400C200A077E1C7FAF12377FC21E25
:10004600E514703690663AE004F0E05407F0E0FFFD
:1000560024FEF582E43462F583E0FE30E71C74FE8C
:100066002FF582E43462F583EE547FF074FE2FF5AB
:1000760082E43462F583E004F514201B2690618344
:10008600E004F0E0543FF0E0FF2467F582E43467D3
:10009600F583E0600ED21B74672FF582E43467F5B2
:1000A60083E4F0201426906619E004F0E0543FF053
:1000B600E0FF24B6F582E43461F583E0600ED214E5
:1000C60074B62FF582E43461F583E4F020152A90A6
:1000D6006184E004F0E05407F0E0FF2408F582E4D0
:1000E6003466F583E0FE30E71074082FF582E434B9
:1000F60066F583EE547FF0D215201303020973E5EB
:100106001554802467F582E43466AF82F53F8F404C
:10011600301D0CC21D200A077E1C7FBD12377F30A2
:10012600160CC216200A077E1C7FC212377F2018C3
:1001360006201903020971854082853F83A3E0FFEB
:10014600906407E0FEEF6E600302096D85408285CC
:100156003F83E0544F24BF603E24FE605414700376
:1001660002028B24FB70030203DD1470030203FDFD
:100176001470030203FD240B600302096D200A07B5
:100186007E1C7FC812377FE50B54E5F53EA2D09260
:100196009B7599E502096D200A077E1C7FD21237EE
:1001A6007FE50B54E5F53EA2D0929B7599E50209D1
:1001B6006D200A077E1C7FDC12377FE50B54E5F5C0
:1001C6003EA2D0929B7599E5854082853F83A3A385
:1001D600E0642D600302096D853F8385408263A23A
:1001E6000190665B63A2017F0A122C61E54024043C
:1001F600F582E4353FF583E0543F6406600302026E
:1002060086E5402408F582E4353FF583E030E74F84
:10021600200A077E1C7FE512377F301E0302096D18
:10022600D21EE4906F4CF0906182F0E5402406F512
:1002360082E4353FF583E014FFC4540F906F4DF010
:10024600EF540FFF25E0FFE5402408F582E4353F33
:10025600F583E0640154012F906F52F002096D207E
:100266000A077E1C7FEE12377F201E0302096D905F
:100276006F4CE06406600302096D7402F002096DBA
:10028600C21E02096D200A077E1C7FF812377F8581
:100296004082853F83A3A3E0646760030203412095
:1002A6000A077E1D7F0012377F75080AE54024087D
:1002B600F582E4353FF583E0750C00F50DE5402445
:1002C60009F582E4353FF583E0FEE4EE420CE540B5
:1002D600240AF582E4353FF583E0F553E540240B27
:1002E600F582E4353FF583E0F552E540240CF582CE
:1002F600E4353FF583E0F551E540240DF582E4351C
:100306003FF583E0F554E540240EF582E4353FF5EC
:1003160083E0F54FAE0CAF0D7C037DE8121E3D8FDA
:1003260050123550906F4EE558F0A3E557F0A3E50F
:1003360056F0A3E555F0D22002096D854082853F2F
:1003460083A3A3E0642D600302096D853F83854086
:100356008263A20190665B63A2017F0A122C61E5AB
:10036600402404F582E4353FF583E0543F6406708B
:1003760061E5402408F582E4353FF583E0FF30E788
:100386003A301E0302096DD21EE4906F4CF0906F56
:10039600D4F0E5402406F582E4353FF583E014FE0B
:1003A600C4540F906F4DF0EE540FFE25E0FEEF643F
:1003B6000154012E906F52F002096D201E030209AE
:1003C6006D906F4CE06406600302096D7402F002E2
:1003D600096DC21E02096D200A077E1D7F0B1237AA
:1003E6007F906100740BF0906407E0906101F07FEC
:1003F6000212435102096D200A077E1D7F12123731
:100406007FE508C394055005050802096D301C1EDA
:10041600906406E0FF6017906610E0D39F400FE4FB
:10042600F510D212C2992099FDD29902096D201EAB
:1004360003020521906FD4E0FF60686401702E20EE
:100446000A077E1D7F1912377F90665B63A20190B3
:10045600610063A2017F09122C619061007408F0AB
:10046600906104740AF07F09124351802C200A0718
:100476007E1D7F2212377F90665B63A2019061002A
:1004860063A2017F09122C619061007408F09061EB
:10049600047447F07F09124351E4906FD4F0C21EF2
:1004A60002096D906F4CE064057034200A077E1DCA
:1004B6007F2C12377F90665B63A20190610063A276
:1004C600017F09122C619061007408F09061041498
:1004D600F07F09124351906F4C7406F002096D903B
:1004E6006F4CE064037034200A077E1D7F37123795
:1004F6007F90665B63A20190610063A2017F09128F
:100506002C619061007408F090610414F07F091268
:100516004351906F4C7407F002096DE51265117036
:10052600030205F6E5112408F53E74082511F511B8
:10053600D21C9061007408F0906407E0FF9061019E
:10054600F0A3741EF0A37401F0A37403F0A3EFF0FC
:100556007400253EF582E43460F583E0049061067C
:10056600F0E4A3F07401253EF582E43460F583E0FF
:10057600906108F07402253EF582E43460F583E06C
:10058600F5587403253EF582E43460F583E0F557AB
:100596007404253EF582E43460F583E0F55674056F
:1005A600253EF582E43460F583E0F5551231C0AF9F
:1005B600507E007C037DE8121E2B8E0C8F0DEF9073
:1005C6006109F0E50CA3F0A3E553F0A3E552F0A30F
:1005D600E551F0A3E554F0A3E54FF07F1012435127
:1005E600300A0302096D7E1D7F4312377F02096DB3
:1005F600201503020696C2159061007408F09064F7
:1006060007E0FF906101F0A37407F0A37401F0A363
:10061600F0A3EFF0906184E0FDC43354E0049061F0
:1006260006F0E4A3F0ED25E025E0243BF582E43472
:1006360066F583E0906108F0906184E0FF25E0258F
:10064600E0243CF582E43466F583E0906109F0EF3E
:1006560025E025E0243DF582E43466F583E09061EB
:100666000AF0906184E025E025E0243EF582E4343A
:1006760066F583E090610BF0E4A3F07F0D12435121
:10068600300A0302096D7E1D7F4C12377F02096D09
:10069600E51470030207E9200A077E1D7F5812370A
:1006A6007FE51425E025E0F553E4F5149061007428
:1006B60008F0906407E0FF906101F0A37422F0E572
:1006C600532480A3F0A37401F0A3EFF090663AE000
:1006D600FFC43354E0906106F0A37401F075F04056
:1006E600EFA42408F582E5F03464F58363A2019053
:1006F600610863A201AF53122C71E55375F003A490
:100706002408F53E90663AE0FF25E025E0241AF538
:1007160082E43466F583E0F558EF25E025E0241BF6
:10072600F582E43466F583E0F55790663AE0FF25F6
:10073600E025E0241CF582E43466F583E0F556EF07
:1007460025E025E0241DF582E43466F583E0F555C1
:100756001231C0AF507E007C037DE8121E2B8E0C3A
:100766008F0DEFAE3E053E74002EF582E43461F542
:1007760083EFF0E50CFFAE3E053E74002EF582E4F5
:100786003461F583EFF0AF3E053E74002FF582E449
:100796003461F583E553F0AF3E053E74002FF582D4
:1007A600E43461F583E552F0AF3E053E74002FF563
:1007B60082E43461F583E551F0AF3E053E74002FC7
:1007C600F582E43461F583E554F0AF3E053E7400EE
:1007D6002FF582E43461F583E54FF0AF3E124351C5
:1007E60002096D2014030208F8200A077E1D7F67A0
:1007F60012377FC2149061007408F0906407E0FF1E
:10080600906101F0A37425F0A37401F0A3F0A3EFA7
:10081600F0906619E0FF906106F0A37402F0EF25F0
:10082600E025E0F53EFF053E74062FF582E43463CD
:10083600F583E0906108F0AF3E053E74062FF58221
:10084600E43463F583E0906109F0AF3E053E74063B
:100856002FF582E43463F583E090610AF0AF3E053C
:100866003E74062FF582E43463F583E090610BF065
:10087600E4A3F074FC253EF53EFF053E74FE2FF51D
:1008860082E43461F583E0F558AF3E053E74FE2FF1
:10089600F582E43461F583E0F557AF3E053E74FE1C
:1008A6002FF582E43461F583E0F556AF3E053E74DC
:1008B600FE2FF582E43461F583E0F5551231C0AFC1
:1008C600507E007C037DE8121E2B8E0C8F0DEF9060
:1008D600610DF0E50CA3F0A3E553F0A3E552F0A3F8
:1008E600E551F0A3E554F0A3E54FF07F1412435110
:1008F6008075301B5F200A077E1D7F7312377FC20B
:100906001B9061007408F0906407E0FF906101F0AD
:10091600A37409F0A37484F0A37403F0A3EFF0901A
:100926006183E0FF25E025E0906106F0A37401F005
:1009360075F008EFA42408F582E5F03464F58363C6
:10094600A20190610863A2017F04122C717F141228
:10095600435180139061007409F0906407E0906140
:0D09660001F07F02124351C219C218C213E2
:010973002261
:0845A4007E1D7F8312377F2288
:0100220022BB
:103D9B00020974E493A3F8E493A34003F68001F2C1
:103DAB0008DFF48029E493A3F85407240CC8C33329
:103DBB00C4540F4420C8834004F456800146F6DFF8
:103DCB00E4800B01020408102040809045ACE47E97
:103DDB00019360BCA3FF543F30E509541FFEE493ED
:103DEB00A360010ECF54C025E060A840B8E493A3B4
:103DFB00FAE493A3F8E493A3C8C582C8CAC583CADF
:103E0B00F0A3C8C582C8CAC583CADFE9DEE780BE96
:0145B2000008
:101DE500BB010689828A83E0225002E722BBFE02FC
:091DF500E32289828A83E493222F
:101DFE00BB010CE58229F582E5833AF583E022509A
:101E0E0006E92582F8E622BBFE06E92582F8E222E3
:0D1E1E00E58229F582E5833AF583E49322FD
:101E2B00EF8DF0A4A8F0CF8CF0A428CE8DF0A42ECB
:021E3B00FE2285
:101E3D00BC000BBE0029EF8DF084FFADF022E4CC89
:101E4D00F875F008EF2FFFEE33FEEC33FCEE9DEC52
:101E5D00984005FCEE9DFE0FD5F0E9E4CEFD22ED98
:101E6D00F8F5F0EE8420D21CFEADF075F008EF2FE2
:101E7D00FFED33FD4007985006D5F0F222C398FDD3
:051E8D000FD5F0EA2270
:101E9200A3F8E0C5F025F0F0E58215827002158303
:061EA200E0C838F0E82260
:101EA80075F008758200EF2FFFEE33FECD33CDCCF1
:101EB80033CCC58233C5829BED9AEC99E582984074
:101EC8000CF582EE9BFEED9AFDEC99FC0FD5F0D651
:101ED800E4CEFBE4CDFAE4CCF9A88222B800C1B97B
:101EE8000059BA002DEC8BF084CFCECDFCE5F0CBB9
:101EF800F97818EF2FFFEE33FEED33FDEC33FCEBF2
:101F080033FB10D703994004EB99FB0FD8E5E4F9AC
:101F1800FA227818EF2FFFEE33FEED33FDEC33FC99
:101F2800C933C910D7059BE99A4007EC9BFCE99A8D
:101F3800F90FD8E0E4C9FAE4CCFB2275F010EF2FD2
:101F4800FFEE33FEED33FDCC33CCC833C810D707D2
:101F58009BEC9AE899400AED9BFDEC9AFCE899F80D
:0E1F68000FD5F0DAE4CDFBE4CCFAE4C8F922A0
:0E1F7600C3E49FFFE49EFEE49DFDE49CFC227C
:101F8400EB9FF5F0EA9E42F0E99D42F0EC6480C8D4
:061F940064809845F02274
:101F9A00EB9FF5F0EA9E42F0E99D42F0E89C45F09D
:011FAA002214
:101FAB00E493FC740193FD740293FE740393FF227C
:101FBB00E493F8740193F9740293FA740393FB227C
:0C1FCB00ECF0A3EDF0A3EEF0A3EFF02289
:101FD700A8828583F0D083D082121FEE121FEE12E3
:101FE7001FEE121FEEE473E493A3C583C5F0C58308
:101FF700C8C582C8F0A3C583C5F0C583C8C582C854
:0120070022B6
:0C200800A42582F582E5F03583F58322E3
:102D38008B3D8A3E893FE4F549F548F547F546F568
:102D480044F545E541454245406012EBC0E0EAC024
:102D5800E0E9C0E0AB40AA41A942122063AB3D05BF
:102D68003FE53FAA3E7002053E14F9121DE5F54AFB
:102D7800C394094007E54AD3940D40E1E54A64202D
:102D880060DBE54AB42D054345038016E54AB42BBC
:102D980005434501800C74FF253FF53F74FF353E20
:102DA800F53EE54360046410703FAB3DAA3EA93F81
:102DB800121DE564306009E543702E75430A8029C9
:102DC800900001121DFEFF64786004EFB4581343AD
:102DD80045017543107402253FF53FE4353EF53E45
:102DE8008007E5437003754308AB3D053FE53FAAFF
:102DF8003E7002053E14F9121DE5F54AC394614080
:102E08000AE54AD3947A5003534ADF74D0254AF529
:102E18004AC3940A400CE54A9411406D74F9254A56
:102E2800F54AE54AD39543506043450185494E85A7
:102E3800484D85474C85464BAF437E00E4FCFDABCF
:102E480049AA48A947A846122014C8ECC8C9EDC920
:102E5800CAEECACBEFCBE4FCFDFEEB254AF549EE02
:102E68003AF548ED39F547EC38F546AF49AE48AD87
:102E780047FCAB4EAA4DA94CA84BD3121F9A50033E
:102E8800022DF1434504022DF1E54520E003E480DD
:102E98002DE54145424540601EAB3DE53F24FFF925
:102EA800E53E34FFFAEBC0E0EAC0E0E9C0E0AB4041
:102EB800AA41A942122063E54530E20774FFFFFEEC
:102EC800FDFC22E545AF49AE48AD47AC4630E103CD
:042ED800021F76223D
:10201400E88FF0A4CC8BF0A42CFCE98EF0A42CFC6B
:102024008AF0EDA42CFCEA8EF0A4CDA8F08BF0A4E9
:102034002DCC3825F0FDE98FF0A42CCD35F0FCEB48
:102044008EF0A4FEA9F0EB8FF0A4CFC5F02ECD390D
:0F205400FEE43CFCEAA42DCE35F0FDE43CFC227A
:10206300BB011A89828A83D0F0D0E0F8D0E0F9D09E
:10207300E0FAD0E0FBE8C0E0C0F00220BB5016E974
:10208300F8D083D082D0E0F9D0E0FAD0E0FBC08270
:10209300C0830220B2BBFE16E9F8D083D082D0E021
:0F20A300F9D0E0FAD0E0FBC082C0830220C42253
:0920B200EBF608EAF608E9F62253
:0920BB00EBF0A3EAF0A3E9F02226
:0920C400EBF208EAF208E9F2224D
:00000001FF
